:100000000C945C020C94A0020C94A0020C94A0022C
:100010000C94A0020C94A0020C94A0020C94A002D8
:100020000C94A0020C94A0020C94970C0C94690DF3
:100030000C94D61B0C94A0020C94A0020C94A00269
:100040000C94A0020C94A0020C94A0020C94A002A8
:100050000C94A0020C943D1C0C94A0020C94A002E1
:100060000C94A0020C94A0020C94A0020C94A00288
:100070000C94A0020C94A0020C94A0020C94A00278
:100080000C94A0020C94A0020C94A0020C94A00268
:100090000C94A0020C94A0020C94A0020C94A00258
:1000A0000C94A0020C94A0020C94A002CE0DF00DB2
:1000B000DB0EF00DDB0E320E550EDB0EAA0EBD0E62
:1000C000CC11CC11FB11FB1146126812CF13CF13C8
:1000D0007312CF131C131C13C013CF13CF13C913E8
:1000E0002913291329132913291329132913291330
:1000F0002913291329132913291329132913291320
:100100003A1348134F13561360130000F0A100C8B0
:1001100001C82E004C002A000030358100001E006E
:10012000140004001D7134004D001F001A00160059
:100130001B00E104C1002000080007000600500079
:100140002C0021001500090019004F004A00220070
:1001500017000A00050000006574500001540000FB
:100160002F7F0000E3004F000154000030770000B3
:10017000E20023001C000B00110000002971240084
:1001800018000D74100052004B0025000C000E00EA
:10019000360051002800260012000F0037002F0003
:1001A0002B81270013003382387130004E002D0060
:1001B0003100347801302D81000001000100010080
:1001C0000100010000003A001E0023002602010089
:1001D00001003B001F0024002702010001003C0039
:1001E000200025002F004B0101003D0021002600CA
:1001F00030004E0101003E002200270027000000D1
:1002000001000100010000000100000001000100E8
:10021000010000000100000001003F000100240275
:10022000310200000100400001002D022202010005
:100230000100410001002D002E00010001004200DC
:10024000010013001F0201000100430001002E0203
:10025000010001000100440045000100010001000F
:100260000000010001000100010001000000010088
:1002700001004B00010001000100010001004A00E3
:10028000010001000100010001004D00010001001A
:100290000100010001004E00010001000100010009
:1002A0000100010001000000010001000100000048
:1002B0000100000001000100010000000100000039
:1002C0000100010001000100010000000100010027
:1002D000010001000100A90001000100010001006E
:1002E000AC00AA00B600010001000100AB00A800AC
:1002F00001000100010001000100010001000100F6
:100300000100AE000100010000001603450072006C
:1003100067006F0044006F007800200045005A001D
:10032000000016034500720067006F0044006F0074
:100330007800200045005A00000004030904090267
:100340006D00040100A0FA0904000001030101008E
:10035000092111010001223F000705810308000A5D
:100360000904010001030102000921110100012219
:100370004D000705820308000A090402000103007A
:10038000000009211101000122360007058303083E
:10039000000A090403000103000000092111010003
:1003A0000122390007058403100001120110010029
:1003B000000008EDFE07130100010200010501091C
:1003C00006A101050719E029E71500250195087523
:1003D000018102050819012905950575019102950C
:1003E000017503910105071900297715002501956D
:1003F0007875018102C005010980A10185021601FD
:100400000026B7001A01002AB70075109501810077
:10041000C0050C0901A1018503160100269C021AE2
:1004200001002A9C02751095018100C00501090296
:10043000A1010901A10005091901290515002501DE
:10044000950575018102950175038101050109304A
:1004500009311581257F95027508810609381581B6
:10046000257F950175088106050C0A38021581253E
:100470007F950175088106C0C005010906A1010527
:100480000719E029E71500250195087501810295F6
:100490000175088101050819012905950575019166
:1004A000029501750391010507190029FF15002523
:1004B000FF950675088100C011241FBECFEFDAE05A
:1004C000DEBFCDBF04B603FE24C08091F20190913F
:1004D000F301A091F401B091F5018730904BA74052
:1004E000B04BB9F41092F2011092F3011092F401A2
:1004F0001092F50114BE84B7877F84BF88E10FB6E0
:10050000F89480936000109260000FBEE0E0FFE37B
:10051000099511E0A0E0B1E0EAEEF7E402C0059031
:100520000D92A433B107D9F711E0A4E3B1E001C003
:100530001D92A23FB107E1F70E94DF090C94F3235B
:100540000C940000CF93DF93EC01662319F0613027
:1005500079F031C08A818823C9F082E00E94561167
:100560008D81982F907F71F080FD0CC086E21BC0BA
:100570008A818823D9F082E00E9456118D81982FBC
:10058000907F71F48D818F708D8315C08D81807FF8
:1005900019F086E20E94071182E00E945D110BC0F3
:1005A00080FDF0CF87E20E943F1005C08D81807FE3
:1005B00099F387E2EFCF80E090E0DF91CF9108954B
:1005C00008956091B1017091B2018091B301909151
:1005D000B4010E943D1B56985E9825982D98269848
:1005E0002E9827982F98813019F0823021F00895A5
:1005F000259A2D9A0895269A2E9A08950C94E10230
:1006000056985E9825982D9826982E9827982F987A
:100610008FEF90E0909389008093880090938B00F7
:1006200080938A0090938D0080938C00259A2D9A58
:100630002FEF80E792E0215080409040E1F700C02A
:100640000000269A2E9A2FEF80E792E021508040FA
:100650009040E1F700C00000279A2F9A2FEF80E723
:1006600092E0215080409040E1F700C000002598C2
:100670002D982FEF80E792E0215080409040E1F7E5
:1006800000C0000026982E982FEF80E792E02150BE
:1006900080409040E1F700C0000027982F985698BE
:1006A0005E9825982D9826982E9827982F9808952B
:1006B00089EA8093800089E08093810024982C98B7
:1006C0003F988AB18F748AB96E98479A8BB1806BC4
:1006D0008BB9769A0E9400030C94E00280E280932A
:1006E00000018091340181110EC00E94BD0381E0A0
:1006F000809334012FEF83ED90E3215080409040B0
:10070000E1F700C0000080E40E94C3038093000171
:1007100081112EC00E94ED0380930001811128C039
:100720000E94ED0380930001811122C08FE30E949B
:10073000ED038093000181111BC00E94E50380E45A
:100740000E94C30380930001811112C08CE00E94BB
:10075000ED038093000181110BC00E94ED03809393
:100760000001811105C08FE30E94ED038093000119
:100770000E94E5038091000108951092B9008AE07B
:100780008093B800089594EA9093BC009091BC00C7
:1007900097FFFCCF9091B900987F983021F090316D
:1007A00011F081E008958093BB0084E88093BC0041
:1007B0008091BC0087FFFCCF8091B900887F883191
:1007C00011F0803471F780E0089584E98093BC00D3
:1007D0008091BC0084FDFCCF08958093BB0084E829
:1007E0008093BC008091BC0087FFFCCF9091B90042
:1007F000987F81E0983209F480E0089584E880933E
:10080000BC008091BC0087FFFCCF8091BB000895A5
:1008100080910001811115C080E40E94C303809380
:10082000000181110CC082E10E94ED038093000160
:10083000811105C08FEF0E94ED03809300010E949B
:10084000E50384B1807F84B985B1807F85B98AB1A1
:10085000837F8AB98BB1837F8BB93E984698089580
:100860000E946E03809300010E94080480B38C7084
:1008700080BB81B3836F81BBE4E4F1E0A6E3B1E028
:1008800011921D9281E0E235F807D1F70C945803DC
:10089000BF92CF92DF92EF92FF920F931F93CF936D
:1008A000DF9380910001882379F0809135018F5F7B
:1008B00080933501811108C00E946E03809300016E
:1008C000811102C00E94000306E311E0C0E0D0E005
:1008D000DD24D39482E0C82EEE24E394F12CC730BB
:1008E00000F580910001811162C080E40E94C30381
:1008F00080930001811112C082E10E94ED03809378
:10090000000181110BC0C7010C2E01C0880F0A9491
:10091000EAF780950E94ED03809300010E94E503B1
:1009200046C0CA30A1F028F4C83059F0C93061F08F
:1009300005C0CC3089F070F0CD3089F0209A28982D
:1009400010C0219A29980DC0229A2A980AC0239A89
:100950002B9807C0529A01C0539A5B9802C03E9AE6
:100960004698E0EAEA95F1F78FB179995AC092E09A
:1009700081708D25892B7C9B02C090E001C094E0A2
:10098000892B7D9B02C090E001C098E0892B7E9B63
:1009900002C090E001C090E1892B9FB19095991F12
:1009A0009927991F9295990F907E892B0FC080915E
:1009B000000181114BC080E40E94C30380930001B9
:1009C000882389F1B12C0E94E5038B2DF8019081D9
:1009D000981719F08083C09201010E9408042196A3
:1009E0000F5F1F4FCE30D10509F079CF8091010103
:1009F000882371F1815080930101882339F08FE9B8
:100A00009FE00197F1F700C0000022C0A4E4B1E02C
:100A1000E6E3F1E081918D9391E0E434F907D1F7B9
:100A200017C090E0A5CF83E10E94ED038093000101
:100A30008111C8CF81E40E94C3038093000181111A
:100A4000C1CF0E94FE03B82EB094BDCF80E0BECFD0
:100A50000E94FE0281E0DF91CF911F910F91FF90E4
:100A6000EF90DF90CF90BF900895E82FF0E0EC5B1F
:100A7000FE4F808108950895089596E0799FF001D2
:100A8000112494E5899FE00DF11D1124E60FF11D5D
:100A9000EE0FFF1FEE5EFE4F859194910895880F33
:100AA000991F86579040FC01859194910895880F75
:100AB000991F865F9E4FFC018591949108950F9335
:100AC0001F93CF93DF93EC01811520E3920730F55C
:100AD000811530E2930708F0B1C08B3B910588F493
:100AE000883A910508F058C0853A910508F049C048
:100AF0008430910508F043C08130910509F4C2C1EA
:100B0000BEC18F3F910509F0D0F5803F910508F0F7
:100B100092C0805E9109089790F1B1C1C11581E53D
:100B2000D807A8F4C23090E5D90708F09FC0C115D6
:100B300020E5D20709F486C008F092C0C11580E410
:100B4000D80708F09CC18E011127106CDCC1C115BB
:100B500090E8D90758F4C11520E7D20708F08BC1F7
:100B6000C11530E6D30708F423C189C1C11580E956
:100B7000D80708F084C18E011F70106AC4C18E01AD
:100B8000C2C1853A910509F480C1863A910509F4FC
:100B90007FC103E810E4B7C1883A910509F47BC12D
:100BA000893A910509F47AC18A3A910509F479C123
:100BB0008B3A910509F478C18C3A910509F477C113
:100BC0008D3A910509F476C1803B910509F475C110
:100BD0008E3A910509F474C18F3A910509F473C1F5
:100BE000813B910509F472C1823B910509F471C101
:100BF000833B910509F470C1843B910509F46FC1F1
:100C0000853B910509F46EC1863B910509F46DC1E0
:100C1000873B910509F46CC1883B910509F46BC1D0
:100C2000893B910509F46AC18A3B910509F069C1C4
:100C30000AE216E468C18C01106565C19F700E94CC
:100C4000570562C10E9419149FEF24E33CE09150C4
:100C500020403040E1F700C000000E94621C53C1F8
:100C60008091D30181608093D3014DC10E940A1EFF
:100C7000811102C00E94F01D0E94271E90E09093F7
:100C8000F2018093F101C23080E5D80721F4809110
:100C9000F101816086C0C43090E5D90721F48091CC
:100CA000F10182607EC0C63020E5D20721F4809138
:100CB000F101846076C0C83030E5D30719F4809123
:100CC000F10127C0CA3080E5D80721F48091F101F5
:100CD000806167C0CC3090E5D90721F48091F101A3
:100CE00080625FC0CE3020E5D20721F48091F1010F
:100CF000806457C0C03130E5D30721F48091F10101
:100D000080684FC0C23180E5D80729F48091F10195
:100D10008460886046C0C33090E5D90721F4809193
:100D2000F1018E7F3EC0C53020E5D20721F48091CD
:100D3000F1018D7F36C0C73030E5D30721F48091B3
:100D4000F1018B7F2EC0C93080E5D80719F480915E
:100D5000F10126C0CB3090E5D90721F48091F10153
:100D60008F7E1FC0CD3020E5D20721F48091F101A4
:100D70008F7D17C0CF3030E5D30721F48091F1018A
:100D80008F7B0FC0C13180E5D80721F48091F1013C
:100D90008F7707C0C331D04531F48091F1018B7F4B
:100DA000877F8093F1018091F1010E942B1EABC0DF
:100DB0008D2F99278F70992781309105E9F48E0145
:100DC000037011279C0102C0220F331F0A95E2F71E
:100DD00089011C68CE01E4E0880F991FEA95E1F7CC
:100DE00088279370082B192BF3E0CC0FDD1FFA95A1
:100DF000E1F7C076DD272CC08230910529F41C2F45
:100E00000027016F106A7FC08330910561F4CE0125
:100E10008370992701E010E002C0000F111F8A952E
:100E2000E2F71C680EC084309105A9F4CE018370EE
:100E3000992701E010E002C0000F111F8A95E2F728
:100E40001A6863E0CC0FDD1F6A95E1F7C07ED770AA
:100E50000C2B1D2B58C08530910529F41C2F002721
:100E6000046F106A50C0069709F04DC0CF71DD279E
:100E70001C2F002702C08E011F70106244C000E0CA
:100E800010E041C001E010E03EC001E810E43BC0CA
:100E900002E810E438C002EE14E435C009EE14E4B0
:100EA00032C00AEE14E42FC005EB14E42CC006EBAC
:100EB00014E429C007EB14E426C00CEC14E423C0AE
:100EC0000DEC14E420C003E815E41DC00AE815E4A5
:100ED0001AC002E915E417C004E915E414C001E2E0
:100EE00016E411C003E216E40EC004E216E40BC0DF
:100EF00005E216E408C006E216E405C007E216E4BF
:100F000002C000E014E4C801DF91CF911F910F915E
:100F1000089596E0799FF001112494E5899FE00DF2
:100F2000F11D1124E60FF11DEE0FFF1FEE5EFE4FC7
:100F300085919491803E9105E0F4803C910558F5AF
:100F40008133910509F46FC048F48932910509F4A1
:100F500063C08A32910509F46DC072C0893391056E
:100F6000E9F082389105D1F08533910509F44DC03F
:100F700067C0833E910581F138F4803E9105B9F058
:100F8000823E9105D9F05CC0863E910561F1873EB5
:100F90009105A1F155C00E944F0508952091F101DE
:100FA00020FD02C021FF4CC080EE90E049C080913E
:100FB000F10180FFF9CF89E390E042C08091F10117
:100FC00082FF0EC08091F10184FF03C080E090E0B9
:100FD00037C083EE90E034C08091F10182FFF2CF00
:100FE00082EE90E02DC08091F10183FF0BC08091D3
:100FF000F10184FDEBCF87EE90E022C08091F101FA
:1010000083FFF5CF86EE90E01BC08091F10185FF54
:1010100007C089E290E014C08091F10185FFF9CF0B
:1010200085E390E00DC08091F10186FF07C08AE260
:1010300090E006C08091F10186FFF9CF81E390E056
:101040000E945F05089508950C9423088091620121
:101050000895CF93DF9300D01F92CDB7DEB72091D4
:10106000E801243019F523E029839B838A832093A8
:10107000E9008FEF9091E800815095FD06C095ED55
:101080009A95F1F700008111F5CF8091E80085FF76
:101090000DC040E050E063E070E0CE0101960E9498
:1010A0008A0A8091E8008E778093E8000F900F9075
:1010B0000F90DF91CF910895CF93DF9300D01F92CF
:1010C000CDB7DEB72091E801243021F522E0298355
:1010D0009B838A8383E08093E9008FEF9091E800FF
:1010E000815095FD06C095ED9A95F1F700008111AC
:1010F000F5CF8091E80085FF0DC040E050E063E04F
:1011000070E0CE0101960E948A0A8091E8008E77F5
:101110008093E8000F900F900F90DF91CF9108958A
:101120002091E8012430F1F422E02093E9002FEF30
:101130003091E800215035FD06C035ED3A95F1F7C4
:1011400000002111F5CF2091E80025FF0BC040E001
:1011500050E065E070E00E948A0A8091E8008E7796
:101160008093E8000895CF93DF93EC018091E8012C
:10117000843009F046C090910C019923D9F09091E8
:101180000D019923B9F08093E9008FEF9091E80069
:10119000815095FD06C095E19A95F1F70000811107
:1011A000F5CF8091E80085FF2CC040E050E060E181
:1011B00070E017C081E08093E9008FEF9091E80024
:1011C000815095FD06C095ED9A95F1F700008111CB
:1011D000F5CF8091E80085FF14C040E050E068E062
:1011E00070E0CE010E948A0A8091E8008E77809399
:1011F000E80080E1FE01A2E5B1E001900D928A9540
:10120000E1F7DF91CF9108958091E701811109C045
:101210000E941C0C0E94790C8091E20084608093F3
:10122000E20008951092E7010895089508950C943E
:10123000D01B42E061EC81E00E94960B42E061EC41
:1012400082E00E94960B42E061EC83E00E94960BE4
:1012500042E161EC84E00C94960B8091EA018330CA
:1012600009F455C030F4813071F0823009F48EC039
:1012700008958A3009F47AC08B3009F460C089304F
:1012800009F09CC020C08091E901813A09F096C024
:101290008091E800877F8093E8008091ED01909134
:1012A000EE01892B21F060E080E090E003C060E176
:1012B00082E591E070E00E94D30A8091E8008B778C
:1012C0008093E80008958091E901813209F076C0A9
:1012D0008091ED019091EE01009719F0039709F0CC
:1012E0006DC08091E800877F8093E8008091E800DE
:1012F00082FD05C08091E8018111F8CF5FC0809127
:10130000F100809362018091E8008B7753C0809157
:10131000E901813A09F052C08091ED019091EE010E
:10132000892B09F04BC08091E800877F8093E8000B
:101330008091E80080FFFCCF80910C0136C0809145
:10134000E9018132D9F58091ED019091EE01892B6F
:10135000A9F58091E800877F8093E8000E94CB0B7D
:101360008091EB0180930C010C9419148091E90198
:10137000813221F58091E800877F8093E8000E9408
:10138000CB0B8091EC018093630108958091E9017A
:10139000813AA1F48091E800877F8093E8008091F2
:1013A000E80080FFFCCF809163018093F100809181
:1013B000E8008E778093E8000C94CB0B089584B7F7
:1013C000877F84BF88E10FB6F89480936000109205
:1013D00060000FBE90E080E80FB6F8948093610043
:1013E000909361000FBE0E94650F0E941C0C0E942A
:1013F000790C8091E20084608093E20078940E94EE
:10140000F40E0E94670F82E091E00E94110F80911C
:10141000E801853069F40E94901B8091E6018823E1
:10142000B1F30E94BB1B882391F30E94740AEFCF93
:101430000E946D0FECCF292F332723303105A9F0FF
:101440006CF42130310509F442C02230310509F035
:1014500043C08DE690E02EE333E042C021323105F7
:10146000C9F02232310519F137C099278130910531
:1014700041F08230910541F0892B71F5EAE3F3E008
:1014800005C0E2E2F3E002C0EAE0F3E0849190E01C
:101490009F0126C0643000F5E62FF0E0EE0FFF1F3D
:1014A000EE5DFE4F2081318189E090E019C064300B
:1014B00098F4E62FF0E0DF01AA0FBB1FA65EBE4F37
:1014C0002D913C91EA5EFE4F808190E009C082E15F
:1014D00090E02BEA33E004C080E090E020E030E0D0
:1014E000FA0131832083089580E189BD82E189BDBD
:1014F00009B400FEFDCF8091D8008F7D8093D80085
:101500008091E00082608093E0008091E00081FDA6
:10151000FCCF0895CF92DF92EF92FF920F931F932B
:10152000CF93DF937C018B01EA010E94EC0B8111C8
:1015300031C0209731F088819981081B190BE80E82
:10154000F91EC12CD12C0115110519F18091E8006B
:1015500085FD14C08091E8008E778093E800209785
:1015600041F0888199818C0D9D1D9983888385E048
:1015700011C00E94EC0B882331F30CC0F70181915C
:101580007F018093F10001501109FFEFCF1ADF0AAC
:10159000DACF80E0DF91CF911F910F91FF90EF9014
:1015A000DF90CF9008952091EF013091F001261740
:1015B000370748F06115710539F42091E8002E775E
:1015C0002093E80001C0B901FC0120E0611571051C
:1015D000B9F18091E801882309F440C0853009F40D
:1015E0003FC08091E80083FD3DC08091E80082FF0C
:1015F00006C08091E80082FF26C080E008958091B7
:10160000E80080FFE3CF2091F3008091F20090E0AA
:10161000922B6115710551F08830910538F42191B4
:101620002093F100615071090196F3CF21E00897F2
:1016300009F020E08091E8008E778093E800C6CF23
:101640002111C7CFD6CF8091E801882339F08530AA
:1016500039F08091E80083FFCCCF04C082E0089588
:1016600083E0089581E008952091EF013091F00129
:101670002617370748F06115710539F42091E80005
:101680002E772093E80001C0B901FC0120E061152C
:101690007105C1F18091E801882309F441C08530CA
:1016A00009F440C08091E80083FD3EC08091E800CD
:1016B00082FF06C08091E80082FF27C080E0089585
:1016C0008091E80080FFE3CF2091F3008091F20049
:1016D00090E0922B6115710559F08830910540F426
:1016E00024912093F1003196615071090196F2CF57
:1016F00021E0089709F020E08091E8008E77809340
:10170000E800C5CF2111C6CFD5CF8091E80188234D
:1017100039F0853039F08091E80083FFCBCF04C0E9
:1017200082E0089583E0089581E00895982F97302E
:1017300058F59093E900981739F07091EC002091DA
:10174000ED005091F00003C0242F762F50E021FFD0
:1017500019C03091EB003E7F3093EB003091ED00EB
:101760003D7F3093ED003091EB0031603093EB0022
:101770007093EC002093ED005093F0002091EE0068
:1017800027FF07C09F5FD3CF8F708093E90081E070
:10179000089580E008958091E90187FD05C080915A
:1017A000E80080FF0EC012C08091E80082FD05C0F5
:1017B0008091E8018111F8CF08958091E8008B773E
:1017C00008C08091E8018111EACF08958091E80076
:1017D0008E778093E80008958091E4009091E50071
:1017E00045E62091EC0020FF21C02091E80020FD7B
:1017F00021C02091E801222389F0253089F0209131
:10180000EB0025FD0FC02091E4003091E500281782
:10181000390739F3415041F0C901E3CF82E008951F
:1018200083E0089581E0089584E008952091E80020
:1018300022FFDFCF80E008950E948A0C0E94920C64
:10184000E0EEF0E0808181608083E8EDF0E080816F
:101850008F77808319BCA7EDB0E08C918E7F8C933D
:1018600080818F7E80831092E70108950F931F93EC
:10187000CF93DF930E948A0C0E94920CC8EDD0E0B7
:1018800088818F77888388818068888388818F7D2D
:10189000888319BC1092E8011092E4011092E601CD
:1018A0001092E50100EE10E0F80180818B7F8083CB
:1018B00088818160888342E060E080E00E94960B2E
:1018C000E1EEF0E080818E7F8083E2EEF0E08081C7
:1018D00081608083808188608083F80180818E7F31
:1018E0008083888180618883DF91CF911F910F91E0
:1018F0000895E8EDF0E080818F7E8083E7EDF0E0F1
:1019000080818160808384E082BF81E08093E701F1
:101910000C94360CE8EDF0E080818E7F808310928D
:10192000E20008951092DA001092E10008951F92EB
:101930000F920FB60F9211242F933F934F935F9303
:101940006F937F938F939F93AF93BF93EF93FF9387
:101950008091E10082FF0BC08091E20082FF07C00E
:101960008091E1008B7F8093E1000E94F30E8091D3
:10197000DA0080FF1FC08091D80080FF1BC08091DB
:10198000DA008E7F8093DA008091D90080FF0DC04D
:1019900080E189BD82E189BD09B400FEFDCF81E00F
:1019A0008093E8010E94040905C019BC1092E80167
:1019B0000E9412098091E10080FF19C08091E2002D
:1019C00080FF15C08091E2008E7F8093E2008091BD
:1019D000E20080618093E2008091D8008062809371
:1019E000D80019BC85E08093E8010E941609809117
:1019F000E10084FF30C08091E20084FF2CC080E1D0
:101A000089BD82E189BD09B400FEFDCF8091D80077
:101A10008F7D8093D8008091E1008F7E8093E100DC
:101A20008091E2008F7E8093E2008091E2008160ED
:101A30008093E2008091E401882311F084E007C0E4
:101A40008091E30087FF02C083E001C081E08093C2
:101A5000E8010E9417098091E10083FF29C080916D
:101A6000E20083FF25C08091E100877F8093E10041
:101A700082E08093E8011092E4018091E1008E7F82
:101A80008093E1008091E2008E7F8093E20080915C
:101A9000E20080618093E20042E060E080E00E942A
:101AA000960B8091F00088608093F0000E941509E9
:101AB000FF91EF91BF91AF919F918F917F916F9126
:101AC0005F914F913F912F910F900FBE0F901F90FC
:101AD00018951F920F920FB60F9211242F933F93D8
:101AE0004F935F936F937F938F939F93AF93BF9326
:101AF000CF93EF93FF93C091E900CF708091EC00FA
:101B00001092E9008091F000877F8093F000789434
:101B10000E94A50D1092E9008091F00088608093EA
:101B2000F000C093E900FF91EF91CF91BF91AF9189
:101B30009F918F917F916F915F914F913F912F91E5
:101B40000F900FBE0F901F9018951F93CF93DF93A8
:101B5000CDB7DEB7AA970FB6F894DEBF0FBECDBFE4
:101B6000E9EEF1E08091F100819321E0E13FF2079D
:101B7000C9F70E942D098091E80083FF1CC12091C4
:101B8000E9013091EA01832F90E08A30910508F055
:101B900012C1FC01EA5AFF4F0C94A323203881F0B4
:101BA000223809F008C18091ED018F708093E9001F
:101BB0008091EB0085FB882780F91092E90006C030
:101BC0008091E5019091E601911182609091E80089
:101BD000977F9093E8008093F1001092F100C5C0C8
:101BE000822F8D7F09F0E7C0222319F0223061F0A7
:101BF000E2C08091EB01813009F0DDC0333009F0A3
:101C000080E08093E60128C08091EB01811124C01F
:101C10002091ED012F7009F4CEC02093E90080914E
:101C2000EB0080FF19C08091EB00333011F480622B
:101C300011C080618093EB0081E090E0022E01C032
:101C4000880F0A94EAF78093EA001092EA008091E4
:101C5000EB0088608093EB001092E9008091E8002F
:101C6000877F86C02111A7C01091EB011F7780915B
:101C7000E3008078812B8093E3008091E800877FE8
:101C80008093E8000E94CB0B8091E80080FFFCCF9E
:101C90008091E30080688093E300112311F083E0DA
:101CA00001C082E08093E80186C02058223008F00D
:101CB00082C08091EB019091EC018C3D23E0920772
:101CC00079F583E08A838AE289834FB7F894DE014D
:101CD000139620E03EE051E2E32FF0E050935700EE
:101CE000E49120FF03C0E295EF703F5FEF708E2F0D
:101CF00090E0EA3010F0C79601C0C0968D939D9396
:101D00002F5F243149F74FBF8091E800877F809390
:101D1000E8006AE270E0CE0101960E94D30A14C086
:101D2000AE014F5F5F4F6091ED010E941B0A00976B
:101D300009F441C02091E800277F2093E800BC010E
:101D400089819A810E94340B8091E8008B7780937F
:101D5000E80031C0203879F58091E800877F8093D2
:101D6000E8008091E4018093F1008091E8008E7793
:101D70008093E8000E94CB0B1EC021111CC09091E3
:101D8000EB019230C0F48091E800877F8093E800F7
:101D90009093E4010E94CB0B8091E401811104C077
:101DA0008091E30087FF02C084E001C081E080935E
:101DB000E8010E9419098091E80083FF0AC0809120
:101DC000E800877F8093E8008091EB008062809339
:101DD000EB00AA960FB6F894DEBF0FBECDBFDF9121
:101DE000CF911F9108950895CF938091E8018823A2
:101DF000B1F08091E9008F709091EC0090FF02C0EB
:101E000090E801C090E0C92FC82B1092E9008091A2
:101E1000E80083FD0E94A50DCF70C093E900CF912B
:101E2000089590936901809368010895E091680195
:101E3000F0916901309721F00190F081E02D099433
:101E400080E00895E0916801F0916901309721F0F8
:101E50000280F381E02D09940895E0916801F091EA
:101E60006901309721F00480F581E02D09940895EF
:101E700020916601309167018217930771F090936A
:101E8000670180936601E0916801F09169013097E4
:101E900021F00680F781E02D0994089520916401D6
:101EA000309165018217930771F0909365018093DB
:101EB0006401E0916801F0916901309721F000849C
:101EC000F185E02D0994089508950C94640F0E9403
:101ED000FF1B0E9430040C94C51CCF92DF92EF923E
:101EE000FF920F931F93CF93DF93CDB7DEB72B975E
:101EF0000FB6F894DEBF0FBECDBF0E9448043BE68C
:101F0000E32E31E0F32E00E010E0C02E802F0E947F
:101F10003505F701D1907F01D826B1F40F5F1F4F2F
:101F20000E30110591F78FEF89838A831B820E94FF
:101F3000081C8160782F9D838C8349815A816B8135
:101F40008D810E94101041C09091D30191FF04C077
:101F50008B870E943B058B8520E030E04D2D50E0C3
:101F6000922FBA01022E02C0759567950A94E2F786
:101F700060FF25C02E83CF82EE24E394F12C02C0B3
:101F8000EE0CFF1C9A95E2F790E08E219F2121E054
:101F9000892B09F420E028870E94081C8160782F93
:101FA0009A8789874E815F8168858A850E94101093
:101FB000F801E559FE4F80818E25808306C02F5F92
:101FC0003F4F2630310561F6A9CF0E94A91F10911D
:101FD0006A010E94160F1817A1F00E94160F809335
:101FE0006A012B960FB6F894DEBF0FBECDBFDF910E
:101FF000CF911F910F91FF90EF90DF90CF900C94B5
:1020000024082B960FB6F894DEBF0FBECDBFDF912C
:10201000CF911F910F91FF90EF90DF90CF90089597
:10202000CF93DF93CDB7DEB72B970FB6F894DEBF13
:102030000FBECDBF4F83588769877A878B87DE01B4
:10204000119686E0FD0111928A95E9F785E0FE017F
:10205000379601900D928A95E1F749815A816B81FB
:102060007C818D819E810E94E9162B960FB6F89493
:10207000DEBF0FBECDBFDF91CF9108950895CF93FE
:10208000C82F882309F4C1C0823859F40E94160F62
:1020900081FDBBC089E30E94301A0E94071B89E3BF
:1020A0000CC0833879F40E94160F80FDAEC083E522
:1020B0000E94301A0E94071B83E50E94701ACF917C
:1020C0000C94071B843859F40E94160F82FD9DC0A2
:1020D00087E40E94301A0E94071B87E4EECF8CEF42
:1020E0008C0F813A48F48C2F0E94D52181118DC02C
:1020F0008C2F0E94301AE3CF80E28C0F883048F496
:10210000C77081E001C0880FCA95EAF70E94B41A2F
:10211000D6CF8BE58C0F833078F4C53A29F0C63AD8
:1021200031F482E890E005C081E890E002C083E8E5
:1021300090E0CF910C94380F88E58C0F833108F034
:1021400064C0C83A39F1C93A41F1CA3A49F1CB3AC7
:1021500051F1CC3A59F1CD3A61F1C03B69F1CE3A37
:1021600071F1CF3A79F1C13B81F1C23B89F1C33BB7
:1021700091F1C43B99F1C53BA1F1C63BA9F1C73B25
:10218000B1F1C83BB9F1C93BC1F1CA3BC9F58AE21B
:1021900092E038C082EE90E035C089EE90E032C027
:1021A0008AEE90E02FC085EB90E02CC086EB90E0AB
:1021B00029C087EB90E026C08CEC90E023C08DEC2A
:1021C00090E020C083E891E01DC08AE891E01AC049
:1021D00082E991E017C084E991E014C081E292E0C5
:1021E00011C083E292E00EC084E292E00BC085E26F
:1021F00092E008C086E292E005C087E292E002C069
:1022000080E090E0CF910C944E0FCF9108958823F9
:1022100009F44BC0823859F40E94160F81FF45C063
:1022200089E30E94301A0E94071B89E30CC083389F
:1022300071F40E94160F80FF38C083E50E94301AA7
:102240000E94071B83E50E94701A0C94071B8438B8
:1022500059F40E94160F82FF28C087E40E94301AAA
:102260000E94071B87E4EFCF9CEF980F913A58F339
:1022700090E2980F983050F4877091E001C0990F68
:102280008A95EAF7892F0E94BA1ADFCF9BE5980F4B
:10229000933020F480E090E00C94380F885A83311A
:1022A00020F480E090E00C944E0F0895882321F0F4
:1022B0000E94B41A0C94071B0895882321F00E94F1
:1022C000BA1A0C94071B08958F929F92AF92BF92F7
:1022D000CF92DF92EF92FF920F931F93CF93DF93F2
:1022E00000D000D01F92CDB7DEB77C0185E0F701AA
:1022F000DE01119601900D928A95E1F7F701D080E9
:1023000011810281B580B2942FE0B2222381348101
:10231000232B39F01F3F39F481E0FFEFDF1203C0B8
:1023200003C081E001C080E080FD5DC20E94CB1946
:10233000882319F082E00E940E1AC7010E943E1005
:10234000D9821A8369817A81802F0E949119182F6E
:10235000C92E0E9445190E94181801110E94D11A15
:102360000E94291A882379F0002369F080E2810F06
:10237000883048F082E00E940E1A0E94291ADD245B
:10238000D394D82601C0D12CEC2DE295EF70F0E06B
:10239000E05AFF4F0C94A3238C2D807F9C2D9F70BF
:1023A000B92E882319F0B29490EFB922002389F056
:1023B000BB2009F4DAC180E2810F883020F48B2D34
:1023C0000E94B41A03C08B2D0E94C41A0E94071BDE
:1023D000CCC1812F0E940711BB2009F4E0C1105E1F
:1023E0008B2D183018F40E94BA1A02C00E94CA1A23
:1023F0000E94071BD4C18C2D807F9C2D9F70A92E1D
:10240000803219F0A29480EFA822112319F0113024
:1024100049F132C0002391F0BB2091F181E0B81264
:1024200004C08A2D0E94E41ABAC192E0B91228C0F1
:102430000E94ED1A8A2D0E94981922C0BB2079F0C3
:10244000E1E0BE1208C00E94B11A8A2109F4A7C1B6
:102450000E949B1904C0F2E0BF1609F4A0C10E94BB
:10246000ED1A12C0002329F081E08B1508F497C102
:1024700007C0B11094C108C0002321F0B11075C18C
:102480008A2DEFC0B11078C18A2DF1C02C2D269570
:102490002695237030E02115310521F021303105DA
:1024A00061F07DC1002321F0812F9C2D937002C02B
:1024B00080E090E00E94380F72C1002321F0812F4C
:1024C0009C2D937002C080E090E00E944E0F67C187
:1024D000812F002319F00E94B11E02C00E94191F13
:1024E0000E949E1F5CC18C2D837009F04FC00111AA
:1024F00056C1212F229526952770220F220F812F5A
:102500008F70882E912CA12CB12C022E04C0880C27
:10251000991CAA1CBB1C0A94D2F714FF10C06FE0D0
:1025200070E080E090E004C0660F771F881F991F5D
:102530002A95D2F7609570958095909503C060E0DC
:1025400070E0CB012C2D269526952370422F50E06C
:102550004230510569F04330510589F068297929E5
:102560008A299B294130510571F00E943D1817C1FD
:10257000682979298A299B290E94571810C10E942D
:102580003D18C501B4010E94231809C1002319F0A8
:102590008C2D817001C08695882309F400C1212FFC
:1025A000229526952770220F220F812F8F70882E5B
:1025B000912CA12CB12C022E04C0880C991CAA1CB1
:1025C000BB1C0A94D2F714FF10C06FE070E080E0EB
:1025D00090E004C0660F771F881F991F2A95D2F7D5
:1025E000609570958095909503C060E070E0CB0198
:1025F0002C2D269526952370422F50E04230510510
:1026000069F04330510589F0682979298A299B2985
:102610004130510571F00E941119C1C06829792912
:102620008A299B290E942B19BAC00E941119C50141
:10263000B4010E94F718B3C0412F50E0FA01E05EE8
:10264000F109E531F10508F08BC0E059FF4F0C941A
:10265000A3231F708C2D8F71002331F00E949018DE
:10266000812F0E9456119BC00E94B118812F0E9499
:102670005D1195C0002339F0B11091C08C2D8F7180
:102680000E94D6188CC091E09B1508F488C0F6CF44
:10269000002339F08C2D8F710E94901880C0002388
:1026A000C9F38C2D8F710E94B11879C0002329F0D5
:1026B0008C2D8F710E947B1872C00E9471186FC0A0
:1026C0000023C9F00E9495190E94BA1A0E94C719E6
:1026D000843029F40E94071A8C2D8F7171C0E1E0BB
:1026E000EB1508F480C01C2D1F71812F0E949018DB
:1026F00063E0812F0EC00E9495190E94B41AF1E088
:10270000FB15D0F40E94071A0E949B1964E08C2DDF
:102710008F710F900F900F900F900F90DF91CF91CE
:102720001F910F91FF90EF90DF90CF90BF90AF90EF
:102730009F908F900C94F71981E00F900F900F905D
:102740000F900F90DF91CF911F910F91FF90EF901D
:10275000DF90CF90BF90AF909F908F900C940E1A07
:10276000002339F0BB2009F495CF812F0E943F1040
:1027700016C0BB2009F495CF812F0E9407110FC00E
:102780004C2D4F70612FC7010E94A2020E94961724
:1027900006C04C2D4F70612FC7010E943C05DD2003
:1027A00011F10E94C71980FD1EC0F70112820E941C
:1027B000C1190E949018C7010E9464110E94C1199A
:1027C0000F900F900F900F900F90DF91CF911F916E
:1027D0000F91FF90EF90DF90CF90BF90AF909F90C0
:1027E0008F900C94B1180F900F900F900F900F9046
:1027F000DF91CF911F910F91FF90EF90DF90CF90DD
:10280000BF90AF909F908F9008950E94D11A0E9420
:10281000E11A0E94A31A0E94071B0E944A200E94EC
:102820009E1F80E090E00E94380F80E090E00C94C2
:102830004E0F0E94C11A0C9405140E948619292F6C
:1028400022952F7030E02C3031054CF42A303105C0
:102850006CF42250310922303105B0F407C02C301D
:10286000310571F02F30310559F00EC0803F31F045
:1028700018F4803E48F402C0843F31F481E00895AA
:1028800093FB882780F9089580E00895CF93DF9324
:1028900000D000D01F92CDB7DEB70F900F900F90F1
:1028A0000F900F90DF91CF910895CF93DF9300D0D9
:1028B00000D000D0CDB7DEB726960FB6F894DEBFB5
:1028C0000FBECDBFDF91CF9108951F93CF93DF93BC
:1028D000C091790116E080917A01C81799F0D0E093
:1028E0001C9FF0011D9FF00D1124E558FE4F408103
:1028F000518162817381848195810E945514219652
:10290000C770E9CFDF91CF911F9108954091AB013E
:102910005091AC016091AD017091AE018091AF0119
:102920009091B0010C945514CF938091B001829591
:102930008F7009F05FC08091AD01882309F45AC0FF
:1029400020917901A0917A016091AB017091AC0165
:102950008091AE019091AF0131E06F3F09F030E01E
:10296000B32FC6E02A1709F445C0009721F07F3F36
:1029700021F44B2F03C041E001C040E030E040FDB6
:1029800035C0C29FF001C39FF00D1124E558FE4FE2
:10299000418174132BC04081641328C042814111CE
:1029A00025C0438154814817590710F441505109FB
:1029B000481B590B483C5105C8F48091B0018F70F9
:1029C00080618093B00186E0829FF001839FF00DCB
:1029D0001124E058FE4F80818F70806180838BEAE4
:1029E00091E00E946411CF910C9465142F5F3F4FCA
:1029F0002770B8CFCF910895CF92DF92EF92FF92D8
:102A00000F931F93CF93DF93CDB7DEB762970FB6C7
:102A1000F894DEBF0FBECDBF8C0185E0F801DE016A
:102A20001D9601900D928A95E1F7D8014C9111966F
:102A30005C91119712966C9112971396ED90FC9001
:102A400014977091AB01E091AC012091AE013091EF
:102A5000AF012115310531F0EF3F31F481E07F3FC7
:102A600019F403C081E001C080E0B82FB170CB2E13
:102A700080FD6CC1D090AD01DD2009F4F5C0F0916E
:102A8000B001E216F30638F0C701821B930B883CB5
:102A9000910548F09BC0209530952E0D3F1D283C98
:102AA000310508F093C08F2F807F09F052C0E513E5
:102AB00014C0741312C0D62E61110FC0FF70F061E4
:102AC000F093B0010E9486148BEA91E00E94641199
:102AD0008091B001F80185836CC1EF2831F05F3F30
:102AE00031F481E04F3F19F403C081E001C080E080
:102AF00080FD03C081E0862701C080E0F82FF170DF
:102B0000FF2E80FF1CC08091790120917A0136E070
:102B1000821709F428C190E0389FF001399FF00D29
:102B20001124E558FE4F7181571306C07081471379
:102B300003C07281671303C001968770E9CFD62E58
:102B4000662309F436C18091B00181608093B001A1
:102B500053C0E51308C0741306C0611104C0D80146
:102B60001596FC93AEC04D875E878D859E856A8BDA
:102B70000E941D146A89882329F1D62E662311F13B
:102B80002091B001822F82958F7090E002970CF413
:102B900060C08091AB019091AC0198878F831986BA
:102BA000FB86EA862C87CE01079651C0E51731F1E6
:102BB0004D875E878D859E856A8B0E941D146A896C
:102BC00081112EC0C8010E946411A4C08F2F807F84
:102BD00069F77E2DF98AE88A89890E9446148BEA72
:102BE00091E00E946411EBEAF1E086E0DF011D92C2
:102BF0008A95E9F70E948614D12CDBC07413D8CFD4
:102C00006111D6CFD8011596FC93C8010E946411BA
:102C1000EBEAF1E086E0DF011D928A95E9F7C9C091
:102C2000D62E662379F22091B001822F82958F7083
:102C300090E0029774F08091AB019091AC019A837F
:102C400089831B82FD82EC822E83CE0101960E9435
:102C5000641186E0F801ABEAB1E001900D928A952B
:102C6000E1F70E9494146FC0E216F30628F0C70142
:102C7000821B930B9C0104C0209530952E0D3F1DA7
:102C8000283C310508F052C0D62E662309F49ACFAD
:102C9000E5132CC074132AC08091B00180FD1DC0C3
:102CA000982F92959F70C9F0D80115968C9315971F
:102CB0009F3039F09F5F9295907F8F70892B15968A
:102CC0008C93C8010E94641186E0F801ABEAB1E080
:102CD00001900D928A95E1F736C086E0F801ABEAE3
:102CE000B1E001900D928A95E1F763C04D875E8750
:102CF0008D859E850E941D14882379F086E0F80159
:102D0000ABEAB1E001900D928A95E1F70E9494142C
:102D10000E948614DD24D3944CC08091B001816060
:102D20008093B001C8010E94641143C07E2DF98ACE
:102D3000E88A89890E944614EBEAF1E086E0DF0127
:102D40001D928A95E9F70E94861433C0662309F420
:102D500039CF4D875E878D859E850E941D148823FF
:102D600009F430CFCBCF4D875E878D859E850E943D
:102D70008619292F22952F7030E0223031052CF44E
:102D80009F7041F0811106C00CC0243031052CF435
:102D90009F7049F4805E883020F0C8010E94641161
:102DA000CF2CDC2C06C0D80115969C91907F91F712
:102DB000F8CF8D2D62960FB6F894DEBF0FBECDBF53
:102DC000DF91CF911F910F91FF90EF90DF90CF9007
:102DD00008951F93CF93DF93CDB7DEB72C970FB62F
:102DE000F894DEBF0FBECDBF4F83588769877A87BF
:102DF0008B879C87CE0107960E94FC148823C1F024
:102E00002F8138858A859B85892B31F03F3F11F0D2
:102E100080E003C02F3FE1F781E0811147C04F817F
:102E2000588569857A858B859C850E9455143EC09E
:102E300086E0FE013796DE01119601900D928A958B
:102E4000E1F7FF81E8854A855B854115510531F041
:102E5000EF3F31F481E0FF3F19F403C081E001C08E
:102E600080E080FD23C020917A0130E0C901019605
:102E7000877099276091790170E086179707F1F1C3
:102E8000F983EA835D834C8396E0929FD001939F00
:102E9000B00D1124A558BE4FFE01319601900D9240
:102EA0009A95E1F780937A010E94651416E080916B
:102EB000790190917A01891779F1189FC001112445
:102EC00085589E4F0E94FC14882331F1E0917901CE
:102ED0001E9FF0011124E558FE4F4081518162810F
:102EE0007381848195810E9455148091790190E0CD
:102EF00001968770992780937901D9CF0E94191480
:102F000010927A0110927901EBEAF1E086E0DF019C
:102F10001D928A95E9F7CACF2C960FB6F894DEBFBA
:102F20000FBECDBFDF91CF911F910895EF92FF9219
:102F30000F931F93CF93DF939C01009709F471C007
:102F4000F12CEE24E394E9012196F9018491843770
:102F500040F4843008F056C0813081F0823021F195
:102F600060C0853709F449C0C0F19CE7980F9037DD
:102F700008F057C08F770E94071146C089010E5F85
:102F80001F4FFE01849190E2980F983050F48770A3
:102F9000FE2D01C0FF0F8A95EAF78F2F0E94D41AE9
:102FA00015C00E943F1014C089010E5F1F4FFE0123
:102FB000849190E2980F983068F48770FE2D01C0DC
:102FC000FF0F8A95EAF78F2F0E94DA1A0E94071BDB
:102FD000E8011AC00E940711FBCF2E5F3F4FFE0190
:102FE000C491CC2341F08FE99FE00197F1F700C035
:102FF0000000C150F6CFE90107C0FE01F490E901DD
:10300000229602C00E943F108F2D882341F0EFE9E5
:10301000FFE03197F1F700C000008150F6CF9E012C
:1030200092CFDF91CF911F910F91FF90EF90089574
:1030300008956093B5017093B6018093B7019093A2
:10304000B8010C9405140F931F930091B5011091D2
:10305000B6012091B7013091B801062B172B282B10
:10306000392B0093B5011093B6012093B70130932B
:10307000B8011F910F910C9405140F931F930091A9
:10308000B5011091B6012091B7013091B801062326
:103090001723282339230093B5011093B6012093F9
:1030A000B7013093B8011F910F910C9405140F9341
:1030B0001F930091B5011091B6012091B701309195
:1030C000B80106271727282739270093B501109341
:1030D000B6012093B7013093B8011F910F910C9462
:1030E00005141092B1011092B2011092B301109226
:1030F000B4010C94051441E050E060E070E004C0BD
:10310000440F551F661F771F8A95D2F74093B10170
:103110005093B2016093B3017093B4010C94051401
:1031200041E050E060E070E004C0440F551F661FAE
:10313000771F8A95D2F78091B1019091B201A09149
:10314000B301B091B401842B952BA62BB72B8093A0
:10315000B1019093B201A093B301B093B4010C9468
:10316000051441E050E060E070E004C0440F551FDA
:10317000661F771F8A95D2F7409550956095709598
:103180008091B1019091B201A091B301B091B401CD
:1031900084239523A623B7238093B1019093B20192
:1031A000A093B301B093B4010C94051441E050E036
:1031B00060E070E004C0440F551F661F771F8A95BA
:1031C000D2F78091B1019091B201A091B301B09179
:1031D000B40184279527A627B7278093B101909340
:1031E000B201A093B301B093B4010C9405140F93F2
:1031F0001F930091B1011091B2012091B301309160
:10320000B401062B172B282B392B0093B1011093F7
:10321000B2012093B3013093B4011F910F910C942C
:1032200005140F931F930091B1011091B2012091E9
:10323000B3013091B40106231723282339230093C7
:10324000B1011093B2012093B3013093B4011F91E7
:103250000F910C9405140F931F930091B1011091DD
:10326000B2012091B3013091B40106271727282716
:1032700039270093B1011093B2012093B301309329
:10328000B4011F910F910C9405140895CF92DF9211
:10329000EF92FF920F931F93CF93DF93EC01C090B7
:1032A000B501D090B601E090B701F090B8018091DF
:1032B000B1019091B201A091B301B091B401C82ABB
:1032C000D92AEA2AFB2A0FE110E0B701A601002E55
:1032D00004C076956795579547950A94D2F740FDB7
:1032E00005C00150110988F780E007C0BE01802F9A
:1032F0000E9489070197A9F3802FDF91CF911F9139
:103300000F91FF90EF90DF90CF900895CF93DF93D0
:10331000EC010E944619BE010E948907DF91CF91FE
:103320000895CB010E94861908958091BE010895E9
:103330008093BE0108951092BE0108950E94081C5A
:103340002091BC013091BD018217930750F00E947B
:10335000081C2091BC013091BD01821B930B9C0184
:103360000AC00E94081C2091BC013091BD0120952B
:103370003095280F391F81E0283B3B4008F480E05E
:1033800008958091BB0185958595859508958091D7
:10339000BB01877008950E94081C2091B9013091EB
:1033A000BA018217930768F00E94081C2091B901A6
:1033B0003091BA01821B930B883B9B4078F480E0EC
:1033C00014C00E94081C2091B9013091BA012095C7
:1033D0003095280F391F283B3B4088F38091BB0173
:1033E00082FB882780F991E089278170089598E011
:1033F000899F90011124622B6093BB010E94901859
:103400000E94081C9093BA018093B901089510920C
:10341000BB011092BA011092B90108954091BB010D
:10342000809584238093BB01982F977089F450E096
:10343000282F332727FD30954217530749F08595EC
:10344000859585950E94B1181092BA011092B90124
:1034500008959091BB01977081E009F480E0089590
:1034600090910C019923D9F090910D019923B9F015
:10347000982F9695969596959F3088F5E0910E0138
:10348000F0910F01E90FF11D877021E030E001C0DC
:10349000220F8A95EAF78181822B818308954091DA
:1034A0000E0150910F0120E030E09FEFFA01E20F92
:1034B000F31F6281681799F09F3F19F4611101C0F1
:1034C000922F2F5F3F4F2E30310581F79F3F39F00C
:1034D000FA01E90FF11D97FDFA9582830895089589
:1034E00090910C019923E1F090910D019923C1F085
:1034F000982F9695969596959F3020F5E0910E0120
:10350000F0910F01E90FF11D877021E030E001C05B
:10351000220F8A95EAF72095818128232183089537
:1035200040910E0150910F0120E030E0FA01E20FCE
:10353000F31F9281981301C012822F5F3F4F2E30EC
:103540003105A1F7089581E090E0E0910E01F0913E
:103550000F01E80FF91F1082019680319105A9F73C
:1035600008958091D20108959091D201982B909363
:10357000D201089580959091D20198239093D20121
:1035800008951092D20108959091D101982B9093B3
:10359000D101089580959091D10198239093D10104
:1035A00008951092D10108959091D001982B909395
:1035B000D001089580959091D00198239093D001E7
:1035C00008951092D00108958093BF010E94081CB5
:1035D0009093BD018093BC0108951092BF01109299
:1035E000BD011092BC01089540910E0150910F0150
:1035F00020E030E080E0FA01E20FF31F91819111A9
:103600008F5F2F5F3F4F2F303105A9F70895E0916D
:103610000E01F0910F018091D2018083E0910E01A3
:10362000F0910F0180819091D101892B8083E091ED
:103630000E01F0910F0180819091D001892B808340
:103640008091BF01882399F00E949E1981110E94E8
:10365000ED1AE0910E01F0910F0180819091BF0170
:10366000892B80830E94F41A81110E94ED1A8091A7
:103670000E0190910F010C94220FCF92DF92EF92E6
:10368000FF920F931F936C01EE24FF24C114D10409
:10369000E104F10421F46B017C0180E001C080E1D0
:1036A00033272F2D1E2D0D2D011511052105310557
:1036B00019F0885F6801790197018601A4E03695C9
:1036C000279517950795AA95D1F70115110521059D
:1036D000310519F08C5F6801790197018601F2E0EC
:1036E0003695279517950795FA95D1F70115110588
:1036F0002105310519F08E5F68017901B701A60136
:103700007695679557954795452B462B472B09F09E
:103710008F5F1F910F91FF90EF90DF90CF900895F2
:103720008091E801843021F11092D40120E488E1F5
:1037300090E00FB6F894A895809360000FBE209398
:10374000600080E00E94240883B7817F846083BF8B
:1037500083B7816083BF7894889583B78E7F83BF5A
:1037600088E10FB6F89480936000109260000FBE5D
:10377000089508950895CF930E94B91B0E944804AC
:103780000E94BA1BC0E08C2F0E943505811105C034
:10379000CF5FCE30C1F780E001C081E0CF910895C6
:1037A0000E9419140E94160F0C9424081F920F9265
:1037B0000FB60F9211248F939F93AF93BF93809175
:1037C000D401811113C08091D5019091D601A091AF
:1037D000D701B091D8014196A11DB11D8093D501AB
:1037E0009093D601A093D701B093D801BF91AF9128
:1037F0009F918F910F900FBE0F901F90189582E0B0
:1038000084BD93E095BD9AEF97BD80936E000895B7
:103810002FB7F8948091D5019091D601A091D7014E
:10382000B091D8012FBF0895CF92DF92EF92FF920F
:103830000F931F932FB7F8944091D5015091D60163
:103840006091D7017091D8012FBF6A017B01EE24EE
:10385000FF248C0120E030E0C016D106E206F3061A
:1038600010F441505109481B590BCA011F910F9187
:10387000FF90EF90DF90CF9008951F920F920FB6B8
:103880000F9211248F939F93AF93BF938091D50193
:103890009091D601A091D701B091D8010196A11DB8
:1038A000B11D8093D5019093D601A093D701B09319
:1038B000D801BF91AF919F918F910F900FBE0F9044
:1038C0001F9018950E941C0CF8942FEF87EA91E640
:1038D000215080409040E1F700C0000087E090EB6D
:1038E000DC018093F2019093F301A093F401B09373
:1038F000F5012CE088E190E00FB6F894A89580934C
:1039000060000FBE20936000FFCFEF92FF920F93F5
:103910001F93CF93DF93E82EF12C8F2D0E94350556
:10392000C0E0D0E0082F10E098010C2E02C03595C1
:1039300027950A94E2F720FD05C02196C630D105EF
:1039400099F709C06C2F7F2D80E00E943D05E81299
:10395000F4CF81E005C0F3948EE0F812DECF80E072
:10396000DF91CF911F910F91FF90EF900895CF932A
:10397000C82F8CE20E94851C882321F08C2FCF91C8
:103980000C94851C80E0CF910895CF930E940A1E6D
:10399000811102C00E94F01DC5E6C15049F00E948D
:1039A00048048FE39CE90197F1F700C00000F5CFD0
:1039B00089E20E94B71C811111C18AE20E94B71CE2
:1039C00081110E94F01D85E00E94B71C81110E94A8
:1039D000621C0E94151E8093D30187E00E94B71CD1
:1039E000882399F18BE10E94B71C882351F09091B4
:1039F000D30191FB882780F921E0822780FB91F990
:103A000022C08EE00E94B71C882351F09091D30110
:103A100092FB882780F921E0822780FB92F913C06E
:103A200080E10E94B71C9091D301882341F093FB61
:103A3000882780F921E0822780FB93F904C0892F31
:103A4000809580FB90F99093D3018091D3010E94DF
:103A5000191E0E94271E8093F10180EE0E94B71C60
:103A6000882341F08091F101982F909590FB80F987
:103A70008093F10189E30E94B71C882359F090914B
:103A8000F10191FB882780F921E0822780FB91F9E1
:103A90009093F10182EE0E94B71C882359F0909117
:103AA000F10192FB882780F921E0822780FB92F9BF
:103AB0009093F10186EE0E94B71C882359F09091F3
:103AC000F10193FB882780F921E0822780FB93F99D
:103AD0009093F10183EE0E94B71C882359F09091D6
:103AE000F10194FB882780F921E0822780FB94F97B
:103AF0009093F10185E30E94B71C882359F09091BF
:103B0000F10195FB882780F921E0822780FB95F958
:103B10009093F10181E30E94B71C882359F09091A2
:103B2000F10196FB882780F921E0822780FB96F936
:103B30009093F10181E10E94B71C882359F0909184
:103B4000F10197FB882780F921E0822780FB97F914
:103B50009093F1018091F1010E942B1E8091F1015F
:103B600087FB882780F980930D0187E20E94B71CAC
:103B7000C82F8EE10E94B71C8111C2608FE10E94A4
:103B8000B71C8111C46080E20E94B71C8111C8601B
:103B900081E20E94B71C8111C06182E20E94B71CC1
:103BA0008111C06283E20E94B71C8111C06484E26B
:103BB0000E94B71C882311F0C06802C0CC2329F0F2
:103BC0008C2F0E94221E6C2F03C00E941E1E682F85
:103BD00070E080E090E0CF910C941918CF91089597
:103BE0006DEE7EEF80E090E00E94DD2360E082E0F9
:103BF00090E00E94CB2360E083E090E00E94CB2322
:103C000060E084E090E00E94CB2360E085E090E0FB
:103C10000C94CB2380E090E00E94C52321E08D3EF0
:103C20009E4F09F020E0822F089582E090E00C94EE
:103C3000BD23682F82E090E00C94CB2383E090E0DA
:103C40000C94BD23682F83E090E00C94CB2384E098
:103C500090E00C94BD23682F84E090E00C94CB237B
:103C60008091DB0180FF0BC06091130185E0689FAC
:103C7000B001112475956795759567952AC081FFE8
:103C800009C06091130185E0689FB001112475950A
:103C900067951FC082FF07C06091130185E0689F90
:103CA000B001112416C04091DC014423C9F0609199
:103CB0001201461788F72091130185E0289F900193
:103CC0001124429FC001439F900D112470E00E9477
:103CD0008F236038710540F46115710539F002C019
:103CE00065E070E0862F08958FE7089581E00895DC
:103CF0008091DB0180FF08C06091110170E0759533
:103D000067957595679521C081FF06C06091110187
:103D100070E07595679519C082FF04C0609111012C
:103D200070E010C08091DC018823C1F06091100127
:103D30008617A0F790911101989FC001112470E09F
:103D40000E948F236038710528F46115710521F0F8
:103D5000862F08958FE7089581E0089561E070E06F
:103D6000F4CF803F21F40E94301E819504C0813F32
:103D700029F40E94301E8093DF010895823F21F4D0
:103D80000E94301E819504C0833F29F40E94301E9A
:103D90008093DE010895893F19F40E94781E05C0C2
:103DA0008A3F31F40E94781E81958093E001089546
:103DB0008B3F21F40E94781E819504C08C3F29F42A
:103DC0000E94781E8093E1010895843F21F4809140
:103DD000DD01816017C0853F21F48091DD018260A3
:103DE00011C0863F21F48091DD0184600BC0873FC4
:103DF00021F48091DD01886005C0883F31F4809115
:103E0000DD0180618093DD0108958D3F21F4809173
:103E1000DB0181600BC08E3F21F48091DB01826069
:103E200005C08F3F29F48091DB0184608093DB0122
:103E30000895803F39F48091DF0187FF6CC01092B4
:103E4000DF0169C0813F29F48091DF011816BCF3BE
:103E500062C09091DE01823F29F497FF5CC010920E
:103E6000DE0159C0833F19F41916CCF354C0893FC1
:103E700041F48091E00118160CF04DC01092E00161
:103E80004AC08A3F29F48091E00187FF44C0F6CF01
:103E90008B3F39F48091E10187FF3DC01092E10131
:103EA0003AC08C3F29F48091E1011816BCF333C06D
:103EB000843F21F48091DD018E7F17C0853F21F47E
:103EC0008091DD018D7F11C0863F21F48091DD015D
:103ED0008B7F0BC0873F21F48091DD01877F05C078
:103EE000883F31F48091DD018F7E8093DD0113C026
:103EF0008D3F21F48091DB018E7F0BC08E3F21F43A
:103F00008091DB018D7F05C08F3F29F48091DB011B
:103F10008B7F8093DB018091DE0181110EC0809147
:103F2000DF0181110AC08091E001811106C08091FA
:103F3000E101811102C01092DC0108958DED91E044
:103F40000E942D0F0E94081C9093DA018093D901E2
:103F500008951F93CF93DF938091D9019091DA0157
:103F60000E94141C4091DC01442321F02091140193
:103F700030E006C0209115015AE0259F90011124E0
:103F80008217930708F482C08091DE011091DF014F
:103F9000D091E001C091E101811107C0111105C06C
:103FA000D11103C0CC2309F471C04F3F19F04F5F0A
:103FB0004093DC01181624F40E94301E8093DE0129
:103FC0008091DE0187FF05C00E94301E819580939D
:103FD000DE01111624F40E94301E8093DF018091CF
:103FE000DF0187FF05C00E94301E81958093DF01AD
:103FF0006091DE01662339F11091DF01112319F17F
:10400000772767FD7095872F972F0E94A02223E3C3
:1040100033E343E35FE30E9404230E946D22609335
:10402000DE01612F772767FD7095872F972F0E94FC
:10403000A02223E333E343E35FE30E9404230E94CF
:104040006D226093DF011D1624F40E94781E809378
:10405000E0018091E00187FF05C00E94781E8195F4
:104060008093E0011C1624F40E94781E8093E101E5
:104070008091E10187FF05C00E94781E81958093A1
:10408000E101DF91CF911F910C949E1FDF91CF91A1
:104090001F910895EDEDF1E085E0DF011D928A9515
:1040A000E9F71092DC011092DB010895833081F171
:1040B00028F4813059F08230D1F00895853009F428
:1040C00049C0B8F1863009F456C008952091150111
:1040D000862F90E0820F911D8F3F910520F4620F93
:1040E0006093150108958FEF809315010895209135
:1040F0001401862F90E0820F911D8F3F910520F4CF
:10410000620F6093140108958FEF80931401089556
:1041100020911301862F90E0820F911D8F3F910512
:1041200020F4620F6093130108958FEF80931301C1
:10413000089520911201862F90E0820F911D8F3FEC
:10414000910520F4620F6093120108958FEF809320
:104150001201089520911101862F90E0820F911D88
:104160008F3F910520F4620F6093110108958FEF46
:1041700080931101089520911001862F90E0820F05
:10418000911D8F3F910520F4620F609310010895F7
:104190008FEF809310010895833011F128F481305E
:1041A00049F0823091F00895853081F120F1863018
:1041B000C1F1089580911501681720F4861B809342
:1041C0001501089510921501089580911401681742
:1041D00020F4861B80931401089510921401089511
:1041E00080911301681720F4861B809313010895B2
:1041F00010921301089580911201681720F4861B14
:104200008093120108951092120108958091110176
:10421000681720F4861B80931101089510921101F4
:10422000089580911001681720F4861B8093100177
:1042300008951092100108958B3109F46AC008F5B1
:104240008E3009F470C070F4873009F452C018F44D
:104250008630B9F134C0883009F4A1C08B3009F43C
:104260009EC02DC0813109F479C020F4803109F459
:1042700064C025C0863109F492C0893109F48FC029
:104280001EC0853309F483C060F4873209F47FC00F
:1042900020F48E3108F06DC012C0893209F477C065
:1042A0000EC0833438F48A3308F061C0883309F4CF
:1042B00076C005C0833409F46AC0883461F080E0B8
:1042C00008958091D301817F8E7F8093D30181E017
:1042D0008093E30108950E9419142FEF83ED90E37A
:1042E000215080409040E1F700C000000E94621C15
:1042F00056C09091D301892F8095817080FB90F9F1
:1043000019F09660986027C0997F977F9093D301AA
:1043100046C09091D30191FB882780F921E0822744
:1043200080FB91F913C09091D30192FB882780F90B
:1043300021E0822780FB92F909C09091D30193FB81
:10434000882780F921E0822780FB93F99093D3019D
:10435000882329F191609093D30108950E94191444
:1043600080910D0191E0892780930D0118C027EC01
:1043700001C023EE280F61E070E080E090E004C00F
:10438000660F771F881F991F2A95D2F704C061E036
:1043900070E080E090E00E9419180E94191481E0FA
:1043A000089580E0089580E00895CF93C82F80910C
:1043B000E301813079F018F08230D1F184C0A0910E
:1043C0000E01B0910F018C91813169F0823209F0B8
:1043D0007CC009C0A0910E01B0910F018C91813178
:1043E00011F0823249F48C2F0E94D12181111DC01D
:1043F0008C2F0E941C211AC08C2F0E94D321811166
:1044000014C0C43179F048F4CB3079F0C03109F0F0
:1044100060C082E08093E30108C0C93219F0C8335C
:1044200021F057C01092E30154C081E0817053C065
:10443000C93289F118F5C43171F1A8F4C73009F017
:1044400046C08AE08093150194E19093140193E0B3
:10445000909313018093120188E08093110188E208
:104460008093100134C0CE51C63088F5EC2FF0E0B7
:10447000E65DFE4F80818093E20129C0CE34E9F0F1
:1044800020F4CB3421F56AE013C0C13579F0C23590
:10449000F1F461E00DC08091E201882319F01092DF
:1044A000E20115C081E08093E30115C061E006C020
:1044B0008091E2010E9456200AC06AE08091E201E8
:1044C0000E94CC2004C01092E30180E004C081E08F
:1044D00002C080E0ABCFCF91089504D06894B111B1
:1044E0008DC0089570D088F09F5790F0B92F99270C
:1044F000B751A0F0D1F0660F771F881F991F1AF0EF
:10450000BA95C9F712C0B13081F077D0B1E0089503
:1045100074C0672F782F8827B85F39F0B93FCCF384
:10452000869577956795B395D9F73EF490958095E4
:10453000709561957F4F8F4F9F4F0895E89409C004
:1045400097FB3EF490958095709561957F4F8F4FC6
:104550009F4F9923A9F0F92F96E9BB279395F695DC
:10456000879577956795B795F111F8CFFAF4BB0F5A
:1045700011F460FF1BC06F5F7F4F8F4F9F4F16C0BE
:10458000882311F096E911C0772321F09EE8872F48
:10459000762F05C0662371F096E8862F70E060E004
:1045A0002AF09A95660F771F881FDAF7880F96957D
:1045B000879597F9089557FD9058440F551F59F066
:1045C0005F3F71F04795880F97FB991F61F09F3F00
:1045D00079F087950895121613061406551FF2CF29
:1045E0004695F1DF08C0161617061806991FF1CF79
:1045F00086957105610508940895E894BB276627A0
:104600007727CB0197F908950BD078C069D028F0AF
:104610006ED018F0952309F05AC05FC01124EECF78
:10462000CADFA0F3959FD1F3950F50E0551F629F0D
:10463000F001729FBB27F00DB11D639FAA27F00DFB
:10464000B11DAA1F649F6627B00DA11D661F829F22
:104650002227B00DA11D621F739FB00DA11D621F07
:10466000839FA00D611D221F749F3327A00D611D24
:10467000231F849F600D211D822F762F6A2F112406
:104680009F5750408AF0E1F088234AF0EE0FFF1F59
:10469000BB1F661F771F881F91505040A9F79E3F90
:1046A000510570F014C0AACF5F3FECF3983EDCF3E5
:1046B000869577956795B795F795E7959F5FC1F7CD
:1046C000FE2B880F911D9695879597F9089597F978
:1046D0009F6780E870E060E008959FEF80EC0895A8
:1046E00000240A94161617061806090608950024D1
:1046F0000A9412161306140605060895092E03944B
:10470000000C11F4882352F0BB0F40F4BF2B11F4BE
:1047100060FF04C06F5F7F4F8F4F9F4F089597FBDF
:10472000072E16F4009407D077FD09D00E94A92324
:1047300007FC05D03EF4909581959F4F08957095A4
:1047400061957F4F0895EE0FFF1F0590F491E02DC6
:104750000994AA1BBB1B51E107C0AA1FBB1FA617C8
:10476000B70710F0A61BB70B881F991F5A95A9F71A
:1047700080959095BC01CD010895F999FECF92BD29
:1047800081BDF89A992780B50895A8E1B0E042E08C
:1047900050E00C94E523262FF999FECF92BD81BD00
:1047A000F89A019700B4021639F01FBA20BD0FB66F
:1047B000F894FA9AF99A0FBE08950196272F0E944D
:1047C000CC230C94CB23DC01CB01FC01F999FECF67
:1047D00006C0F2BDE1BDF89A319600B40D92415089
:0A47E0005040B8F70895F894FFCF99
:1047EA0020022608B30890085C0829080101C001C4
:1047FA0028080A03140A3F4D363979042C04F603B3
:10480A00BD035003690382039B03010203040506E7
:04481A000708090082
:00000001FF
